:100000000EC07EC092C026C025C0C6C023C022C07C
:1000100021C020C01FC01EC08AC01CC01BC011242C
:100020001FBECFE5D2E0DEBFCDBF11E0A0E6B0E05D
:10003000E0E8F6E002C005900D92A230B107D9F7D2
:1000400021E0A2E0B1E001C01D92A233B207E1F7C6
:10005000A0D114C36BC0A895F89414BE91B5986153
:1000600091BD813031F0823031F082E481BD7894ED
:10007000089583E4FBCF87E4F9CFA895F89414BEE4
:1000800081B5886181BD11BC7894089585B7877E5C
:10009000806185BFF89485B7806285BF85B7846825
:1000A00085BF8B7F85BF7894889585B78F7D85BF09
:1000B00008950F931F93CF93DF938C01062E000CAE
:1000C000770B85E0660F771F8A95E1F760507040E7
:1000D00040E250E0C801A1D2E801005E1F4F8991C3
:1000E0008C3030F464E670E0F6D084E690E0CDD059
:1000F000C017D107A1F7DF91CF911F910F910895FC
:100100001F921FB61F9211248F93809104018111B9
:1001100007C010920301809127018F5F8093270110
:100120008F911F901FBE1F901895189518958F934B
:100130008FB78F93EF93FF93E2E0F1E081818460CA
:100140008183FF91EF918F918FBF8F9118958AB521
:1001500080688ABD8AB58F7B8ABD089582E089BF99
:1001600083E08ABD81E083BF12BE19BCB89A1092A9
:100170002F0110922C0110922E0110922D0110923D
:100180003101109230011092280110922901109231
:100190002A0110922B0108950F920FB60F921F9211
:1001A00011242F933F934F935F938F939F93AF931C
:1001B000BF93EF93FF9380912F0120912D013091F8
:1001C0002E01820F932F911D90932E0180932D016C
:1001D000E0912D01F0912E01349633E0F695E795EC
:1001E0003A95E1F7EF770E2E000CFF0BEE57FF4F1D
:1001F000808190912C01992309F445C020912C0114
:100200004091300150913101240F352F311D309331
:10021000310120933001E0913001F09131013496A9
:1002200093E0F695E7959A95E1F7EF770E2E000C9F
:10023000FF0BEE57FF4F9081890F96959695891B7E
:1002400089BD8091280190912901A0912A01B09146
:100250002B010196A11DB11D8093280190932901C6
:10026000A0932A01B0932B01FF91EF91BF91AF9121
:100270009F918F915F914F913F912F911F900F9080
:100280000FBE0F90189590E0D7CF109228011092D2
:10029000290110922A0110922B0125B7277E25BF34
:1002A0006FE070E095D1B0E0A0E04091280150915E
:1002B000290160912A0170912B0184179507A607E7
:1002C000B70708F4089525B7206225BF889525B79C
:1002D0002F7D25BFEACFCF93DF93EB011BBE8C3080
:1002E000F0F4E82FEE0FFF0BE659FF4F808180936B
:1002F0002F01818180932C012ADFCE01C6DF8AB5D0
:100300008F778ABD8AB58F7B8ABDC09810922F01E6
:1003100010922C0180E68BBFDF91CF910895863F2C
:1003200031F482E480932F0110922C01E5CF833FBA
:1003300011F481E2F7CF853FB1F482E280932F017F
:1003400010922C0104DFCE0163E070E052D1EB018A
:10035000CB019BDF8BE280932F01CE0196DF83E3FD
:1003600080932F01CACF843F51F683E380932F01FE
:1003700010922C01ECDECE0163E070E03AD1EB018B
:10038000CB0183DF8BE280932F01CE017EDF82E2FF
:10039000E7CF90E896BD16BC88B3866088BB8BE03B
:1003A00080BD98B983E085BF80E68BBF86E085BBC2
:1003B000789481E050DE6ADE60DED0DE10920201C9
:1003C00081E08093040110920301109206011092C3
:1003D0000501E7E0F1E08FEF819391E0E732F90763
:1003E000D9F7FF24F394D1E0CFEF1AE003E026B36E
:1003F000922F927021FB882780F9809304018F153A
:1004000009F4BDC0911122C08091030181608093E5
:1004100003011092270180E01EDE38DEF090040117
:100420008091030180FFB5C082E015DE2FDE809150
:10043000030182FFDCCFD09302018A7F8260809328
:10044000030168EC70E083EF46DFD1CF1092030127
:10045000809127019FEF980F9A3018F0C0932701E1
:10046000DACF912F981B9093270181E0F4DD0EDE07
:1004700004DE8091020181111BC064E670E080916E
:10048000270129DF80910601803240F6E82FF0E055
:10049000EE5FFE4F9091270195838F5F8093060159
:1004A00040E250E060EE70E087E091E0C6D0B6CF69
:1004B000813001F5E091270164E670E08AE0E130E7
:1004C00029F0E23039F464E670E08BE004DF10924A
:1004D0000201A4CF67E0E33049F00E2E000CFF0BC1
:1004E000E05AFF4F6081683008F098CF87E091E0D4
:1004F000E0DD94CF8230C1F4E09127010E2E000C94
:10050000FF0BE05AFF4F808187FDE1CF809305010B
:1005100010920601E7E0F1E0C19381E0E732F807CD
:10052000D9F7009302017ACF833009F077CF809119
:1005300006018032B0F01092020160E273E084EFB5
:10054000CADE60910501683008F068CF70E085E090
:10055000660F771F8A95E1F76050704040E250E0E7
:10056000A3CFE82FF0E0EE5FFE4F90912701958337
:100570008F5F8093060164E670E083EFE1CF9923FB
:1005800009F44CCF1092020110920301C09327018D
:1005900045CF81FF11C082E05EDD78DD80910301EF
:1005A00082FF25CF92E090930201897F809303011F
:1005B00068EC70E085EF48CF85B7877E806185BFA6
:1005C00085B7806285BF889585B78F7D85BF0FCF42
:1005D0000024552704C0080E591F880F991F009743
:1005E00029F076956795B8F37105B9F7802D952FA9
:1005F0000895AA1BBB1B51E107C0AA1FBB1FA6176A
:10060000B70710F0A61BB70B881F991F5A95A9F7BB
:1006100080959095BC01CD010895DC01CB01FC01D2
:10062000E199FECF06C0FFBBEEBBE09A31960DB25A
:100630000D9241505040B8F70895DC01A40FB51F4A
:100640004150504040F0CB01840F951F2E9105D0B2
:1006500041505040D8F70895262FE199FECF9FBB17
:100660008EBBE09A01970DB2021639F01CBA2DBB71
:100670000FB6F894E29AE19A0FBE0895F894FFCF6E
:1006800000FFFFFF010203040506573D4F2E572EC2
:10069000602E4F32573260324F38573860384F3DF6
:1006A000603D404346494C4F5255585B5E6063661F
:1006B000686A6D6F7173757678797B7C7D7E7E7FDD
:1006C0007F7F7F7F7F7F7E7E7D7C7B797876757371
:1006D000716F6D6A686663605E5B5855524F4C4936
:1006E0004643403C393633302D2A2724211F1C191C
:1006F000171512100E0C0A09070604030201010067
:1007000000000000000001010203040607090A0CB2
:100710000E10121517191C1F2124272A2D303336CD
:02072000393C62
:00000001FF
